:0600000080318A2A000095
:0800080083018A012000200899
:10001000A4002108A5002208A6002308A7000B1EA3
:1000200013288B183D282408A0002508A1002608C5
:10003000A2002708A300090021003E082000A1011A
:1000400021003D02031829283D082000A0003B287C
:1000500021002000A00108302100BF00BD0D2000BC
:10006000A00D21003E08200020020318A000A10DD1
:100070002100BF0B2E2820000800A908031D4728D7
:1000800021000C1420000C184628A90AAD282908C4
:10009000083C031C8E2821000C1420000C1C6E2828
:1000A0000D302C07A1002030A3000318A30A21085B
:1000B000840023088500013029022100BB000130A3
:1000C0002000A00021003B082000A10003196B289C
:1000D000A035A10B6828200880048C280D302C073F
:1000E000A1002030A3000318A30A210884002308DC
:1000F0008500013029022100BB0001302000A00052
:1001000021003B082000A10003198928A035A10B7C
:1001100086282008FF3A8005A90AAD2829080A3C4C
:10012000031DAC2801302C072100BC00BD00463067
:10013000BE0020001C202008AC000D302C078400DD
:10014000203085000318850A800121008C102200D0
:100150008C102000A901AD28A90A8B10803113282A
:1001600021008C160C1680312000B92A0830A1001D
:100170000930A000A00BBA2822008C1221008C129A
:1001800008302000A000A00BC3282100BA0D2200D7
:100190000C12031CCE2821000C1622000318D328B1
:1001A00021000C12220021008C1620008C1ED62863
:1001B000A10BB8280930A000A00BDC2822008C126B
:1001C00021008C1200000C1608302000A000A00BAB
:1001D000E7280830A000A00BEB2821008C16200097
:1001E0008C1EF028A1010830A000A00BF5280C1AE5
:1001F000211422008C1221008C1222000C122100EA
:100200000C12200008002100AF08031D0B292E0846
:10021000003C03180E29A830B1001029A030B1000D
:100220000C1609302000A000A00B142921008C1608
:1002300008302000A000A00B1B298C1E1D292200C5
:100240000C1221000C1209302000A000A00B26295E
:1002500022008C1221008C123108BA002000B62036
:1002600021002D08B3002E08B4002F08B500B601F8
:100270002D08BA002000B62021002C08BA0020006A
:10028000B62021000C1609302000A000A00B462942
:1002900021008C1608302000A000A00B4D298C1ED8
:1002A0004F2922000C1221000C1209302000A0005E
:1002B000A00B582922008C1221008C12013031072A
:1002C000B200BA002000B620A00108302100B3001F
:1002D000200020082100B4000C1608302000A000E7
:1002E000A00B702921008C1620008C1E75290C1A79
:1002F00003140C1E0310A10D0930A000A00B7E29D1
:1003000021008C1222008C122100B30B6C290C16D8
:1003100008302000A000A00B8B2922000C12210025
:100320003408031D0C1200008C1620008C1E962928
:100330000930A000A00B9A2922008C1221008C12F7
:1003400008302000A000A00BA32922000C122100DD
:100350000C12200021082100B0000C1200008C16A5
:1003600020008C1EB1290930A000A00BB529B829A6
:10037000000021000C1609302000A000A00BBE29AF
:10038000210030082000A1000800203085005930ED
:10039000840000080319D9290A30A100A001A00B8C
:1003A000CF29A10BCE295F30A000A00BD529800B4F
:1003B000CC298031022B2100B108031DE32930082C
:1003C000003C0318E629A830B400E829A030B400A6
:1003D0000630B4040C1609302000A000A00BEE2952
:1003E00021008C1608302000A000A00BF529220067
:1003F0000C1221000C1209302000A000A00BFE29D5
:1004000022008C1221008C123408BA002000B62081
:1004100021002F08B6003008B7003108B800B90134
:100420002F08BA002000B62021002E08BA002000B4
:10043000B62021003208BA002000B62021000C129C
:1004400000008C1620008C1E232A0930A000A00B6F
:10045000272A2A2A000021000C1609302000A000BB
:10046000A00B302A21000C1609302000A000A00BA0
:10047000372A21008C1608302000A000A00B3E2A4D
:1004800022000C1221000C1209302000A000A00B49
:10049000472A22008C1221008C123408BA00200056
:1004A000B6202108210033102000211C5A2A2100E7
:1004B000331420002100331C882A0C160930200038
:1004C000A000A00B612A21008C1608302000A0009B
:1004D000A00B682A8C1E6A2A22000C1221000C1222
:1004E00009302000A000A00B732A22008C122100EA
:1004F0008C123408BA002000B620210821003310E5
:100500002000211C862A2100331420005A2A2100B1
:1005100020000800850184011F308305F43021008C
:1005200099001A082000A9012A10AB01AC01210092
:10053000A401A301A801A701A601A50123008C0124
:10054000220092019101210017101D101E109E1013
:10055000003023008C008E000B16C0308B04FA3064
:1005600021009900980115138C1022008C14200092
:10057000B0282100AF01AE01AD010330AC00200076
:10058000032121082100A900AF01AE01AD01023015
:10059000AC002000032121082100AA00AF01AE0118
:1005A000AD010130AC002000032121082100AB0087
:1005B000AF01AE01AD01AC012000032121082100F3
:1005C000AC002908A8002A08A7002B08A6002C08C0
:1005D000A500A401A3012000A908031D082B2100E8
:1005E0002408013C0318F62A2000082B031DFE2ACC
:1005F0002308F33C0318FE2A2000082B0130A90031
:100600002000C5292100A30A0319A40AEB2A20000F
:10061000A90803190D2B2100E92A2C082B02031924
:10062000852B21008C1022008C140430210025071A
:10063000A9000030263DAA000030273DAB00003065
:10064000283DAC000D3020002B07840020308500B1
:100650000318850A00082100AD002C08B1002B0802
:10066000B0002A08AF002908AE002D08B200200013
:10067000DB2101302B072100AA002000A8018B1BE1
:10068000A8178B1321002A08BD004630BE002000A9
:100690001C20A81B8B172008AB0001302100A507E8
:1006A0000318A60A0319A70A0319A80A2508A9000E
:1006B000B101B001AF01AE012508B2002000DB217D
:1006C00021002608A900B101B001AF010130AE0040
:1006D0002608B2002000DB2121002708A900B10173
:1006E000B001AF010230AE002708B2002000DB21CC
:1006F00021002808A900B101B001AF010330AE000C
:100700002808B2002000DB210D2B2100E92A63001C
:020000040001F9
:04000E008C39FF1E0C
:00000001FF
